:020000040000fa
:080000001406040000000000da
:020000040000fa
:020000040002f8
:04afe000dfff00008f
:020000040000fa
:020000040002f8
:04afe400ffff00006b
:020000040000fa
:020000040002f8
:04afe80078ff0000ee
:020000040000fa
:020000040002f8
:04afec007dff0000e5
:020000040000fa
:020000040002f8
:04aff00078ff0000e6
:020000040000fa
:1000080000000000000000000000000000000000e8
:100018000c060000000000000000000000000000c6
:10002800000000000000000000000000900900002f
:1000380000000000000000000000000000000000b8
:10004800f60900000000000000000000fa0a0000a5
:10005800660b0000920b000000000000000000008a
:100068000000000000000000000000000000000088
:100078000000000000000000000000000000000078
:10008800000000000000000000000000220a00003c
:100098008e0a0000000000000000000000000000c0
:1000a8000000000000000000000000000000000048
:1000b8000000000000000000000000000000000038
:1000c8000000000000000000000000000000000028
:1000d8000000000000000000000000000000000018
:1000e8000000000000000000000000000000000008
:1000f80000000000000000000000000000000000f8
:1001080000000000000000000000000000000000e7
:1001180000000000000000000000000000000000d7
:1001280000000000320b000000000000000000008a
:1001380000000000000000000000000000000000b7
:1001480000000000000000000000000000000000a7
:100158000000000000000000000000000000000097
:100168000000000000000000000000000000000087
:100178000000000000000000000000000000000077
:100188000000000000000000000000000000000067
:100198000000000000000000be0b0000ea0b000099
:1001a800160c000000000000000000000000000025
:1001b8000000000000000000000000000000000037
:1001c8000000000000000000000000000000000027
:1001d8000000000000000000000000000000000017
:1001e8000000000000000000000000000000000007
:1001f80000000000000000000000000000000000f7
:1002080000000000000000000000000000000000e6
:1002180000000000000000000000000000000000d6
:1002280000000000000000000000000000000000c6
:1002380000000000000000000000000000000000b6
:1002480000000000000000000000000000000000a6
:100258000000000000000000000000000000000096
:100268000000000000000000000000000000000086
:0c0278000000000000000000000000007a
:020000040000fa
:1004000027d2bf002652b7004220af002672ec0070
:1004100027d2d60027d2b60000c0d20027d2bf0014
:1004200000c0fd0027f2b70026d2bf0000c0fd00cb
:100430000040d20027d2b60027d2bf0000c0fd0086
:1004400027f2b7001040b20026f2d60026f2b6001e
:1004500027f2d6003091800000000600803e200088
:10046000030007008100e900fcff3a0000000600dd
:10047000831f7800c20320000400bc006601510005
:10048000e0815900f23fb1000380b1000600350061
:10049000ee03090000000000423fb1000380b100fc
:1004a000fbff3d001200b000223fb000020035000b
:1004b0000280090000000000cf0178000000060063
:1004c000889fbe008a9fbe008c1f78000004be007b
:1004d000850107000478a30026003a006120e100ae
:1004e0002500320009f8a30025003a006420e1004d
:1004f00021003200f507b1000508a3000200320018
:1005000000004000818048006044b80003102000d3
:1005100002002000000040008180480008054400df
:1005200089854c000a0541008b8549000a05500069
:100530008b855800030033000a00be0002047400db
:10054000838474008301d1000281d300830f710082
:10055000f0ff3a008904d1000884d300600149000b
:1005600082017800c1adde00fb07b0007301070017
:10057000070037000960a0000800be000400370033
:100580001202200062918800f0ff2f00f1ff270087
:100590004f0678004f05be004f04be000000060065
:1005a00003f0a200869fbe00889fbe008a9fbe0007
:1005b0008c9fbe0044010700860133006450e100b7
:1005c0004f0032006420e1005200320003826c00d0
:1005d00007003b000905d0000306d000820f54003d
:1005e0000c065d000200390002003200890178002b
:1005f000030678008582550004003d000003fd00dd
:100600008103fd008502ea008b854200840f7200a1
:1006100002003b0060001000e08018006011b8008c
:100620000005eb007a28e1000a0039000600780096
:10063000c75ddd00f707b200878075002d00370029
:10064000828171000a017800610560008180d1001b
:100650000080d3008502e900f9ff3b00060440005a
:100660008784480002003b0060041400e0841c0002
:100670000988a300070032008a817100828171001d
:10068000610164008904d1000884d3008b05e8006f
:10069000170037000978a30013003a000b00e000b0
:1006a000130034008b05e9000804440089844c00e1
:1006b0000a4474000978a3000d003a000b00e00022
:1006c000070034008b05e9000804440089844c00cd
:1006d00001003a000b0020000978a300f7ff320068
:1006e0000001eb0002003700828171000a017800ee
:1006f000120107000cf0a70001f0a0003e01370036
:100700006420e10002003a00838f6c003f01330057
:100710000801be000200be0037013700869fbe0000
:10072000889fbe008a9fbe008c9fbe00e600070027
:100730002801330003866c006450e1002e00320073
:100740006420e100330032006150e1002f003200ec
:100750006120e1003100320085855500eb07b000d3
:1007600009002000080420000500370008044400a8
:1007700089844c000a0031000603430087834b0044
:100780000001530081815b00f8ff33000203be00cb
:100790000800a0000804440089844c00f6ff3900da
:1007a000c639dd0083017300010032001300200010
:1007b0008904d1000884d3000998a3000500320001
:1007c0000800a7000300a0008904d1000884d3001a
:1007d0008b05e8008904d1000884d3000001eb00f8
:1007e0000281d200d500070001f0a1000cf0a700a3
:1007f00001f0a000000137006420e1000301320095
:100800000801be000200be00f7ff37006120e100d2
:10081000fe0032006000b800f3ff37000000200047
:1008200001f82700f0ff3700869fbe00889fbe00ba
:100830008a9fbe008c9fbe00a3000700e500330026
:1008400003866c006450e100240032006420e10063
:10085000270032006150e100220032006120e100f7
:10086000210032008b854200eb07b1000134b80053
:10087000003ab8000804420089844a00013ab800ee
:100880000030b8008880400009014a0004003300ad
:100890000000400081804800020149008b05e9000a
:1008a000c909dd008301700001003200130020003f
:1008b000c814de004814dd004709de001200b20053
:1008c000c808de00088470009c00070001f0a10049
:1008d0000cf0a70001f0a000c70037006120e10084
:1008e000ca0032000801be000200be00f7ff370058
:1008f0006150e100fcff3a00c4003700829fbe0057
:100900000001be00780007000470a70003f0a100fa
:100910006509b100180032000e0035006828e100ba
:1009200007003500f0ff2f00f1ff27000300e00073
:1009300015003b00010028004f01be00000005002b
:1009400000004000818048008502e900fcff3a0079
:1009500009003700f88f420003003c008000eb00e4
:100960004f01be00000005008100d1000080d300cf
:100970008502e800fcff3a000300e00002003b00b3
:1009800060001000e08018004f01be00000006006b
:10099000829fbe000001be00530007000470a70044
:1009a00003f0a10003f8a30015003a006509b100a7
:1009b000110032000a0035006928e100030035000b
:1009c000010028004f01be000000050000004000ab
:1009d000818048008502e900fcff3a0006003700ec
:1009e000f88f4200060035008100d1000080d3005e
:1009f0008502e800fcff3a004f01be00000006003f
:100a00008000eb004f01be00000005000080fb00ed
:100a10008000eb00829fbe00889fbe008a9fbe00c0
:100a2000010578000100e0000400350008003c00ea
:100a30000000e000200032000500370060001000d8
:100a4000e080180002003b0001f024001a0037008b
:100a50000004be006011b8006b0920000982cf00bd
:100a6000020039000882cf000441b0006942520000
:100a70000e00320008003b008281710061016400b9
:100a80008904d1000884d3008b05e8000442e80003
:100a9000f9ff3a00050037000804440089844c003f
:100aa0008b05e9000442e900fbff3a002300070040
:100ab0000af0a70001f0a0004f05be004f04be00e1
:100ac0004f01be00000006000004be000600070043
:100ad0000003be000405be000200be0002000700c5
:100ae000844f750000000600c70ade00f107b2005f
:100af000f50fb20008003200e1cf420002003200e0
:100b00000170a00024000500810f70000100320078
:100b10000408050044000500810f700002003a003f
:100b2000140005008502e9000000400081c0480073
:100b3000fcff3b000170a0002400050081002000a4
:100b4000618055000b003d000b00200061fe2f006e
:100b50000100e1001d003400828171006101640028
:100b60008904d1000884d3000000e800faff3a00ad
:100b7000710020006100640003007000020060004a
:100b80000900320061044400e0844c000988a5009b
:100b9000050032008b05e8006808e10002003a0019
:100ba0008904d1000884d300f20f20000258e1002c
:100bb00005003d00c75ddd00f907b20089807500c2
:100bc00008007800000006000bf827008b00780072
:100bd000000005000200be006450e1000500360080
:100be0006420e100020036000968a30001003a0019
:100bf0000800be000160a0004f06be004f05be0009
:100c00004f04be004f03be0000000600f0ff2f009f
:100c1000f1ff2700f8ff37000020ef000220ef006f
:100c2000c088a900004006000f002100b02e21005e
:100c300000018800000000000000eb0000077800c1
:100c40000c000900002f78000007eb005420ef0093
:100c50000e2eef001e2eef000000eb00a121210060
:100c6000e51d09008018780010cea90010cea9005b
:100c700014cea90010aea90010aea90014aea900b0
:100c800040a7a900a1002000f4fd0700e002200019
:100c9000303a880044e7a90044c7a9004407a900e6
:100ca0004427a9004447a9004467a9004487a90034
:100cb000300020000600fc00317420008207200074
:100cc000a309200082487800834878008048780093
:100cd000113a8000618070000600fc002174200041
:100ce0006204200073052000824878008348780061
:100cf000804878004427ef00e0022000303a880066
:100d0000300020000d00fc0031742000820720001c
:100d1000a309200082487800834878008048780042
:100d200000002000217420006204200073052000d0
:100d300082487800834878008048780042a7ae0057
:100d4000feff3700813e2000c4fd070010c0b30045
:100d500086e6b70090c2b300c4e6b70000022000e8
:100d600000708800007025008070880010eea900d7
:100d70004188a80041a8a80041c8a90004a1a90071
:100d80000481a90005e1a8000068a9001061a8007d
:100d90001021a90011e1a80011a1a90010a1a8002b
:100da0001081a8000621ef000821ef000ca1ef0040
:100db0000ea1ef004408a8004428a9004448a90057
:100dc0000108a9002108a8001fe1a8001fa1a9008f
:100dd0001ec1a9001ea1a9001e81a9001e61a900b3
:100de0001e21a9004d88a9004da8a8004dc8a80043
:100df0000368a90021e1a80021a1a90020c1a90040
:100e000020a1a9002081a9002021a9004e08a90045
:100e10004e28a8004e48a8000388a9002002a90077
:100e20002022a9002042a90020a2a9002062a90036
:100e30002082a90020e2a9002102a9002122a90004
:100e4000700720004011880022a2a90022c2a90038
:100e500022e2a90021e2a8002182a9004588a90078
:100e600045a8a80045c8a8002168a8002828a8000f
:100e70002bc8a9002be8a9002c08a9000bc8a900c1
:100e80000be8a9000c08a90001eca90001aca9001d
:100e9000016ca900014ca900012ca900010ca900ba
:100ea00000eca900008ca90000aca90000cca900ae
:100eb000000ca900002ca900004ca900006ca9009e
:100ec000202cef00402cef00602cef0000202000d1
:100ed00020608800020ca900022ca900024ca90085
:100ee000262cef00462cef00662cef00282cef009c
:100ef000482cef00682cef000aacef0023eca800b0
:100f000023cca90043eca80043cca90063eca800c3
:100f100063cca900dabc2a001b32240030002c006c
:100f2000fa608800fb60880020618800dabc2a0033
:100f30001b32240000002800fa608800fb60880053
:100f400010618800dabc2a001b32240030002c001b
:100f5000fa608800fb60880020628800dabc2a0002
:100f60001b32240000002800fa608800fb60880023
:100f700010628800dabc2a001b32240030002c00ea
:100f8000fa608800fb60880020638800dabc2a00d1
:100f90001b32240000002800fa608800fb608800f3
:100fa0001063880011eea90011aea900116ea9000e
:100fb000a70037003f0037000020200000618800b4
:100fc00000202000006288000020200000638800cc
:100fd000020ca900022ca800024ca80004acef00ef
:100fe00028acef0048acef0068acef00262cef0017
:100ff000462cef00662cef000aacef0023eca800b3
:1010000023cca90043eca80043cca90063eca800c2
:1010100063cca900dabc2a001b32240030002c006b
:10102000fa608800fb60880020618800dabc2a0032
:101030001b32240000002800fa608800fb60880052
:1010400010618800dabc2a001b32240030002c001a
:10105000fa608800fb60880020628800dabc2a0001
:101060001b32240000002800fa608800fb60880022
:1010700010628800dabc2a001b32240030002c00e9
:10108000fa608800fb60880020638800dabc2a00d0
:101090001b32240000002800fa608800fb608800f2
:1010a0001063880011eea90011aea900116ea9000d
:1010b000670037003500370000102000006188000d
:1010c00000102000006288000010200000638800eb
:1010d000020ca900022ca800024ca8000a2cef0068
:1010e00004acef00282cef0050552500406288002a
:1010f000a0aa2a0040638800dabc2a001b32240020
:1011000030002c00fa608800fb60880020618800b5
:10111000dabc2a001b32240000002c00fa60880090
:10112000fb60880010618800dabc2a001b322400b2
:1011300030002c00fa608800fb6088002062880084
:10114000dabc2a001b32240000002c00fa60880060
:10115000fb60880010628800dabc2a001b32240081
:1011600030002c00fa608800fb6088002063880053
:10117000dabc2a001b32240000002c00fa60880030
:10118000fb608800106388003100370030003700b2
:10119000001020000061880000102000006288001c
:1011a000020ca900022ca800024ca8000a2cef0097
:1011b00004acef00282cef000000240040628800ff
:1011c000dabc2a001b32240030002c00fa608800b0
:1011d000fb60880020618800dabc2a001b322400f2
:1011e00000002c00fa608800fb6088001061880015
:1011f000dabc2a001b32240030002c00fa60880080
:10120000fb60880020628800dabc2a001b322400c0
:1012100000002c00fa608800fb60880010628800e3
:10122000dabc2a001b32240030002c00fa6088004f
:10123000fb60880020638800dabc2a001b3224008f
:1012400000002c00fa608800fb60880010638800b2
:10125000218ca900418ca900618ca900216ca900f6
:10126000416ca900616ca900214ca900414ca90066
:10127000614ca90020eca80040eca80060eca8009c
:101280003e2cef005e2cef007e2cef0001eca8005e
:101290000000eb00c14d2100ff00090080587800dc
:1012a000b972ef00ba72ef00a032ef00a232ef0085
:1012b0002e32ef000080eb00014d210005000900f7
:1012c000801878004a32ef004c32ef004e32ef00c7
:1012d000c90707009f070700e00707005232ef0029
:1012e00060a38000e090880070a380001c12b5000d
:1012f000e090880070a380001091880080a3800097
:101300002212b5001c12b4004200de008092880058
:101310005432ef005632ef005832ef0066013700ca
:10132000ff3ffc004200f8003600f8004400f800df
:101330008e1f78000e0020000d000900be1f7800ef
:101340003200f8000100fc000068a9000021ef0055
:101350005412e20006003a008094800010088800d1
:1013600015eea80010002000a0928800140037009d
:10137000a1928000e18f500003003a00200020007d
:10138000a09288000e003700a1928000e28f5000ea
:1013900007003a00f09480009212b500100888000f
:1013a00015eea90030002000a0928800040037004c
:1013b000a1928000e38f500001003a005432ef0008
:1013c000ff3ffc003200f900ae0120000d000900d3
:1013d0004f1778004f0778004400f9003600f900f5
:1013e0004200f9000100fc0000400600ff3ffc0045
:1013f0004200f8003600f8004400f8008e1f780024
:101400000e0020000d000900be1f78003200f80019
:101410000100fc000108a900ff3ffc003200f900b8
:10142000ae0120000d0009004f1778004f0778002b
:101430004400f9003600f9004200f9000100fc0008
:1014400000400600ff3ffc004200f8003600f800b4
:101450004400f8008e1f78000e0020000d000900e7
:10146000be1f78003200f8000100fc000368a900ec
:101470001421ef005612e20006003a00a09480000a
:10148000d008880015aea80010002000b092880097
:1014900017003700b1928000e18f500003003a003e
:1014a00020002000b092880011003700b192800027
:1014b000e28f500007003a00f09480009612b500c9
:1014c000d008880015aea90030002000b092880036
:1014d00007003700b1928000e38f500004003a000b
:1014e000f09480009612b500d00888005632ef00c4
:1014f000ff3ffc003200f900ae0120000d000900a2
:101500004f1778004f0778004400f9003600f900c3
:101510004200f9000100fc0000400600ff3ffc0013
:101520004200f8003600f8004400f8008e1f7800f2
:101530000e0020000d000900be1f78003200f800e8
:101540000100fc000388a9001821ef005812e200f6
:1015500006003a00c0948000e0088800156ea800dc
:1015600010002000c092880017003700c192800050
:10157000e18f500003003a0020002000c092880054
:1015800011003700c1928000e28f500007003a003e
:10159000f09480009a12b500e0088800156ea9004a
:1015a00030002000c092880007003700c192800000
:1015b000e38f500004003a00f09480009a12b500c6
:1015c000e00888005832ef00ff3ffc003200f900cd
:1015d000ae0120000d0009004f1778004f0778007a
:1015e0004400f9003600f9004200f9000100fc0057
:1015f00000400600ff3ffc004200f8003600f80003
:101600004400f8008e1f78000e0020000d00090035
:10161000be1f78003200f8000100fc000168a9003c
:10162000b972ec00b9d2bf008080fb00301180009d
:10163000c24d210080707900ff3ffc003200f900ac
:10164000ae0120000d0009004f1778004f07780009
:101650004400f9003600f9004200f9000100fc00e6
:1016600000400600ff3ffc004200f8003600f80092
:101670004400f8008e1f78000e0020000d000900c5
:10168000be1f78003200f8000100fc000828a90005
:101690002242ae00000037002222af002222a90021
:1016a000ff3ffc003200f900ae0120000d000900f0
:1016b0004f1778004f0778004400f9003600f90012
:1016c0004200f9000100fc0000400600ff3ffc0062
:1016d0004200f8003600f8004400f8008e1f780041
:1016e0000e0020000d000900be1f78003200f80037
:1016f0000100fc000188a900ff3ffc003200f90056
:10170000ae0120000d0009004f1778004f07780048
:101710004400f9003600f9004200f9000100fc0025
:1017200000400600ff3ffc004200f8003600f800d1
:101730004400f8008e1f78000e0020000d00090004
:10174000be1f78003200f8000100fc0001a8a900cb
:10175000ff3ffc003200f900ae0120000d0009003f
:101760004f1778004f0778004400f9003600f90061
:101770004200f9000100fc0000400600ff3ffc00b1
:101780004200f8003600f8004400f8008e1f780090
:101790000e0020000d000900be1f78003200f80086
:1017a0000100fc000bc8a900ff3ffc003200f9005b
:1017b000ae0120000d0009004f1778004f07780098
:1017c0004400f9003600f9004200f9000100fc0075
:1017d00000400600ff3ffc004200f8003600f80021
:1017e0004400f8008e1f78000e0020000d00090054
:1017f000be1f78003200f8000100fc000be8a900d1
:10180000ff3ffc003200f900ae0120000d0009008e
:101810004f1778004f0778004400f9003600f900b0
:101820004200f9000100fc0000400600ff3ffc0000
:101830004200f8003600f8004400f8008e1f7800df
:101840000e0020000d000900be1f78003200f800d5
:101850000100fc000c08a900ff3ffc003200f90069
:10186000ae0120000d0009004f1778004f077800e7
:101870004400f9003600f9004200f9000100fc00c4
:1018800000400600bad2bf00b952e30007003200a0
:10189000ba72ec00bad2bf000080fb00c14d21003b
:1018a00060c07800bbf2b70001003700bbf2ef0068
:1018b0000000060000000600300880000095880047
:1018c0004008800010958800eeff070060ccb30050
:1018d000bb52b50006003900e0cfb300bb52b500e3
:1018e0000100390001003700bc72ef0040023700f0
:1018f000bbf2ae0028003700bc72ef0050c8b30046
:10190000bb52e30005003a00bbd2bf00bcf2b700f7
:10191000bdf2ef00bef2ef001e00370050c9b30069
:10192000bb52e30005003a00bbd2bf00bcf2b700d7
:10193000bff2ef00c0f2ef001600370050cab3004c
:10194000bb52e30005003a00bbd2bf00bcf2b700b7
:10195000c1f2ef00c2f2ef000e00370050cbb3002f
:10196000bb52e30005003a00bbd2bf00bcf2b70097
:10197000c3f2ef00c4f2ef000600370050ccb30012
:10198000bb52e30003003a00bbd2bf00bcf2b70079
:10199000c5f2ef0016023700bc52e20002003a0026
:1019a000130237001202370050c8b300bc52e300e4
:1019b0007f003a0000e0ef00bd52e30003003a0070
:1019c000bbd2bf00bdf2b70078003700bbd2bf006a
:1019d000bef2b700e0c4b300bd52e30022003a00fb
:1019e000cc72ef00be52e20002003600be52d400bc
:1019f00063f2b7006212e20013003600ccd2a800f6
:101a00006012ec00e090880010938000e29080006b
:101a10000200e00002003200110009000280d8003c
:101a2000f0938800f0938000029580001395800069
:101a300000004100e08049000001be0082a688004d
:101a400093a6880006003700d0b4ef00d2b4ef00b0
:101a5000262cef002068a9000068a90015eea90057
:101a6000cb32a80050003700f0c4b300bd52e300f1
:101a700022003a00cd72ef00be52e20002003600b2
:101a8000be52d4006df2b7006c12e20013003600b3
:101a9000cdd2a8006a12ec00e0908800609380002c
:101aa000e29080000200e000020032001100090014
:101ab0000280d80030948800309480000295800025
:101ac0001395800000004100e08049000001be0045
:101ad000a2a68800b3a6880006003700d4b4ef00a1
:101ae000d6b4ef00462cef002368a9000368a900d4
:101af00015aea900cb32a8002b00370000c5b300fb
:101b0000bd52e30022003a00ce72ef00be52e20066
:101b100002003600be52d40077f2b7007612e2001f
:101b200013003600ced2a8007412ec00e0908800ba
:101b3000b0938000e29080000200e00002003200da
:101b4000110009000280d800709488007094800011
:101b5000029580001395800000004100e08049005c
:101b60000001be00c2a68800d3a688000600370088
:101b7000d8b4ef00dab4ef00662cef002388a90098
:101b80000388a900156ea900cb32a8000600370013
:101b9000bdd2bf0080407800e1cf500002003a0083
:101ba00010aea90014aea900bdf2ef0090013700fd
:101bb00050c9b300bc52e30053013a0000e0ef000b
:101bc000bf52e30003003a00bbd2bf00bff2b70030
:101bd0004c013700bbd2bf00c0f2b700c052e200d8
:101be0006a003a00e0c4b300bf52e3001e003a00ae
:101bf000cc72ef006212e20013003600ccd2a800d3
:101c00006012ec00e090880010938000e290800069
:101c10000200e00002003200110009000280d8003a
:101c2000f0938800f0938000029580001395800067
:101c300000004100e08049000001be0082a688004b
:101c400093a6880006003700d0b4ef00d2b4ef00ae
:101c5000262cef002068a9000068a90015eea90055
:101c6000cb32a80048003700f0c4b300bf52e300f5
:101c70001e003a00cd72ef006c12e2001300360035
:101c8000cdd2a8006a12ec00e0908800609380003a
:101c9000e29080000200e000020032001100090022
:101ca0000280d80030948800309480000295800033
:101cb0001395800000004100e08049000001be0053
:101cc000a2a68800b3a6880006003700d4b4ef00af
:101cd000d6b4ef00462cef002368a9000368a900e2
:101ce00015aea900cb32a8002700370000c5b3000d
:101cf000bf52e3001e003a00ce72ef007612e200ff
:101d000013003600ced2a8007412ec00e0908800d8
:101d1000b0938000e29080000200e00002003200f8
:101d2000110009000280d80070948800709480002f
:101d3000029580001395800000004100e08049007a
:101d40000001be00c2a68800d3a6880006003700a6
:101d5000d8b4ef00dab4ef00662cef002388a900b6
:101d60000388a900156ea900cb32a8000600370031
:101d7000bfd2bf0080407800e1cf500002003a009f
:101d800010aea90014aea900de003700e0c4b30015
:101d9000bf52e30045003a0001938000c0d2bf006b
:101da0000080fb0001004000e0928800e19280008a
:101db000f0072000808f500002003600f00720005e
:101dc000e0928800cc72ef002068a90015eea9000f
:101dd0005432ef0060a38000d090880050928000c1
:101de0001a12b500209288006295800073958000d9
:101df0002092800006fb07008bfa0700e4fa070038
:101e000080948800809480004412b50090948800eb
:101e10000068a9002068a800262cef00cc12a800ba
:101e2000d0928000e29280000200e00002003200c6
:101e3000110009000280d800d0938800e192800050
:101e400000938000808f50000d00320000938000ce
:101e50005c12b50001e0af000020ee001091880098
:101e6000f0928000129180000200e0000200320037
:101e7000110009000280d800e093880001003700bb
:101e80007c32ef00d0938000029580001395800093
:101e900000004100e08049000001be0082a68800e9
:101ea00093a68800cb32a80095003700f0c4b30099
:101eb000bf52e30045003a0051938000c0d2bf00fa
:101ec0000080fb00010040003093880031938000c7
:101ed000f0072000808f500002003600f00720003d
:101ee00030938800cd72ef002368a90015aea900d9
:101ef0005632ef0070a38000d0908800609280007e
:101f00001a12b50030928800829580009395800067
:101f100030928000befa070043fa07009cfa0700df
:101f2000a0948800a09480004612b500b094880068
:101f30000368a9002368a800462cef00cd12a80072
:101f400020938000329380000200e0000200320003
:101f5000110009000280d80010948800319380009d
:101f600050938000808f50000d003200509380000d
:101f70006612b50001e0af000020ee00109188006d
:101f800020938000129180000200e00002003200e5
:101f9000110009000280d800209488000100370059
:101fa0008432ef0010948000029580001395800029
:101fb00000004100e08049000001be00a2a68800a8
:101fc000b3a68800cb32a8004d00370000c5b3008f
:101fd000bf52e30045003a00a1938000c0d2bf0089
:101fe0000080fb0001004000809388008193800006
:101ff000f0072000808f500002003600f00720001c
:1020000080938800ce72ef002388a900156ea90086
:102010005832ef0080a38000d0908800709280003a
:102020001a12b50040928800a2958000b3958000f6
:102030004092800076fa0700fbf9070054fa070087
:10204000c0948800c09480004812b500d0948800e5
:102050000388a9002388a800662cef00ce12a800f0
:1020600070938000829380000200e0000200320042
:10207000110009000280d8005094880081938000ec
:10208000a0938000808f50000d003200a09380004c
:102090007012b50001e0af000020ee001091880042
:1020a00070938000129180000200e0000200320074
:1020b000110009000280d8006094880001003700f8
:1020c0008c32ef00509480000295800013958000c0
:1020d00000004100e08049000001be00c2a6880067
:1020e000d3a68800cb32a80005003700bfd2bf00be
:1020f00080407800e1cf500001003a0014aea80003
:10210000bff2ef003a00370050cab300bc52e30000
:102110000a003a0000e0ef00c152e30003003a0079
:10212000bbd2bf00c1f2b70003003700bbd2bf0073
:10213000c2f2b700c10207002d00370050cbb30038
:10214000bc52e3000a003a0000e0ef00c352e30093
:1021500003003a00bbd2bf00c3f2b7000300370050
:10216000bbd2bf00c4f2b700c00207002000370096
:1021700050ccb300bc52e30007003a0000e0ef008f
:10218000c552e30003003a00bbd2bf00c5f2b7005e
:10219000ac0207001600370050cdb300bc52e3007c
:1021a00007003a0000e0ef00c652e30003003a00e7
:1021b000bbd2bf00c6f2b700aa0207000c0037006e
:1021c00050ceb300bc52e30009003a0000e0ef003b
:1021d000c752e30003003a00bbd2bf00c7f2b7000a
:1021e00003003700bbd2bf00c8f2b7009a02070055
:1021f000cb32af007102070030c0b300ca52b50045
:1022000058023100029580001395800040958000af
:1022100051958000800f5100818f5900460239008e
:10222000abf2a800ca52e200bd003a00ccd2bf0017
:1022300080407800e1cf50000c003a007832ef0087
:1022400020c0b300ccf2b700d0938000029580008c
:102250001395800000004100e08049000001be00ad
:1022600082a6880093a68800ac003700ccd2bf00bd
:1022700080407800e2cf500043003a00c1938000d4
:10228000e0928000808f50000f0031007832ec0027
:10229000c293800002014100002d210060007900fe
:1022a00030618800d09380000295800013958000f3
:1022b00000004100e08049000001be0082a68800c5
:1022c00093a688002f003700cc72ef00e1928000c7
:1022d00000938000808f500005003a00d0b4ef00da
:1022e000d2b4ef0000938000c0938800250037002f
:1022f00000938000e1928000808f50001100360032
:10230000cc52a800e0928000c0938800c293800065
:1023100002014100002d2100600079003061880039
:10232000e09380000295800013958000000041003a
:10233000e08049000001be0082a6880093a68800c4
:1023400010003700cc72a800e0928000c093880093
:10235000c293800002014100002d2100600079003d
:1023600030618800e0938000029580001395800022
:1023700000004100e08049000001be0082a6880004
:1023800093a6880065003700ccd2bf00804078005b
:10239000e4cf500016003a007832ed00c29380007e
:1023a00002014100002d21006000790030618800a9
:1023b000e0938000029580001395800000004100aa
:1023c000e08049000001be0082a6880093a6880034
:1023d000c193800000938000808f500003003a007a
:1023e000cc72ef00d0b4ef00d2b4ef004b00370056
:1023f000ccd2bf0080407800e8cf500016003a00f1
:102400007832ec00c293800002014100002d2100cf
:102410006000790030618800e093800002958000c0
:102420001395800000004100e08049000001be00db
:1024300082a6880093a68800c19380000093800044
:10244000808f500003003a00cc72ef00d0b4ef0050
:10245000d2b4ef003100370000c4b300cc52e30027
:1024600012003a0000938000c0938800c29380005d
:1024700002014100002d21006000790030618800d8
:1024800000c8b300ccf2b700f09380000295800042
:102490001395800000004100e08049000001be006b
:1024a00082a6880093a688001c00370000c8b300ed
:1024b000cc52e30019003a007812e2000f00360017
:1024c0007832ed00c293800002014100002d21000e
:1024d0006000790030618800f093800002958000f0
:1024e0001395800000004100e08049000001be001b
:1024f00082a6880093a6880008003700cc72ef00ff
:10250000262cef000021ef002068a9000068a90038
:1025100015eea900d0b4ef00d2b4ef00850137006a
:10252000cad2bf0080407800e1cf5000bf003a001f
:10253000cdd2bf0080407800e1cf50000c003a00bf
:102540008032ef0020c0b300cdf2b70010948000bd
:10255000029580001395800000004100e080490052
:102560000001be00a2a68800b3a68800ae00370016
:10257000cdd2bf0080407800e2cf500043003a0047
:102580000194800030938000808f50000f00310054
:102590008032ec000294800002014100002d2100f5
:1025a00060007900306288001094800002958000fd
:1025b0001395800000004100e08049000001be004a
:1025c000a2a68800b3a688002f003700cd72ef00c6
:1025d0003193800050938000808f500005003a00b6
:1025e000cd92a800d4b4ef00d6b4ef005093800091
:1025f000009488005093800031938000808f5000b9
:1026000011003600cd52a80030938000009488005d
:102610000294800002014100002d21006000790039
:10262000306288002094800002958000139580001d
:1026300000004100e08049000001be00a2a6880021
:10264000b3a6880010003700cd72a8003093800038
:10265000009488000294800002014100002d2100b6
:10266000600079003062880020948000029580002c
:102670001395800000004100e08049000001be0089
:10268000a2a68800b3a6880067003700cdd2bf009d
:1026900080407800e4cf500017003a008032ed000f
:1026a0000294800002014100002d210060007900a9
:1026b000306288002094800002958000139580008d
:1026c00000004100e08049000001be00a2a6880091
:1026d000b3a688000194800050938000808f500042
:1026e00004003a00cd52a900cd92a800d4b4ef0066
:1026f000d6b4ef004c003700cdd2bf008040780048
:10270000e8cf500017003a008032ec0002948000bd
:1027100002014100002d2100600079003062880034
:1027200020948000029580001395800000004100f5
:10273000e08049000001be00a2a68800b3a6880080
:102740000194800050938000808f500004003a0074
:10275000cd72a900cd92a800d4b4ef00d6b4ef009a
:102760003100370000c4b300cd52e30012003a003c
:102770005093800000948800029480000201410080
:10278000002d2100600079003062880000c8b3008d
:10279000cdf2b70030948000029580001395800040
:1027a00000004100e08049000001be00a2a68800b0
:1027b000b3a688001c00370000c8b300cd52e30068
:1027c00019003a008012e2000f0036008032ed005e
:1027d0000294800002014100002d21006000790078
:1027e000306288003094800002958000139580004c
:1027f00000004100e08049000001be00a2a6880060
:10280000b3a6880008003700cd72ef00462cef0019
:102810001421ef002368a9000368a90015aea900e0
:10282000d4b4ef00d6b4ef00c2003700cad2bf0064
:1028300080407800e2cf5000be003a00ced2bf0008
:1028400080407800e1cf50000c003a008832ef0061
:1028500020c0b300cef2b7005094800002958000f3
:102860001395800000004100e08049000001be0097
:10287000c2a68800d3a68800ae003700ced2bf0023
:1028800080407800e2cf500043003a00419480003d
:1028900080938000808f50000f0031008832ec0060
:1028a0004294800002014100002d21006000790067
:1028b000306388005094800002958000139580005a
:1028c00000004100e08049000001be00c2a688006f
:1028d000d3a688002f003700ce72ef0081938000ce
:1028e000a0938000808f500005003a00ce92a8008f
:1028f000d8b4ef00dab4ef00a093800040948800d1
:10290000a093800081938000808f500011003600da
:10291000ce52a800809380004094880042948000aa
:1029200002014100002d2100600079003063880021
:1029300060948000029580001395800000004100a3
:10294000e08049000001be00c2a68800d3a688002e
:1029500010003700ce72a800809380004094880059
:102960004294800002014100002d210060007900a6
:102970003063880060948000029580001395800089
:1029800000004100e08049000001be00c2a68800ae
:10299000d3a6880067003700ced2bf008040780001
:1029a000e4cf500017003a008832ed0042948000d6
:1029b00002014100002d2100600079003063880091
:1029c0006094800002958000139580000000410013
:1029d000e08049000001be00c2a68800d3a688009e
:1029e00041948000a0938000808f500004003a0042
:1029f000ce52a900ce92a800d8b4ef00dab4ef000e
:102a00004c003700ced2bf0080407800e8cf5000a5
:102a100017003a008832ec00429480000201410025
:102a2000002d2100600079003063880060948000f0
:102a3000029580001395800000004100e08049006d
:102a40000001be00c2a68800d3a688004194800081
:102a5000a0938000808f500004003a00ce72a9003d
:102a6000ce92a800d8b4ef00dab4ef0031003700fe
:102a700000c4b300ce52e30012003a00a0938000dd
:102a8000409488004294800002014100002d210002
:102a9000600079003063880000c8b300cef2b70050
:102aa0007094800002958000139580000000410022
:102ab000e08049000001be00c2a68800d3a68800bd
:102ac0001c00370000c8b300ce52e30019003a00e2
:102ad0008812e2000f0036008832ed004294800038
:102ae00002014100002d2100600079003063880060
:102af00070948000029580001395800000004100d2
:102b0000e08049000001be00c2a68800d3a688006c
:102b100008003700ce72ef00662cef001821ef009e
:102b20002388a9000388a900156ea900d8b4ef0076
:102b3000dab4ef0021000700a3f2ae00080037006e
:102b4000a032ef00a232ef000621ef000821ef00d3
:102b50000080eb00014d210005000900801878007d
:102b600006003700a3f2ae0004003700a032ef00e9
:102b7000a232ef000621ef000821ef0020f6070047
:102b8000d0908800e09480001a12b60080918800ee
:102b9000e0948000e09088001c32d5008091800095
:102ba0001c12b500f0948800a212af0014eea80029
:102bb000a212ae0014eea9003ffb3700caf2ef00ec
:102bc000abf2a800c972ef0020c0b300c952e30005
:102bd00018003e00c9d2bf000080fb00c200dd002b
:102be000004d2100008040001000be000001be002a
:102bf0004095800051958000800f5100818f5900d1
:102c00000a003100c9d2bf000080fb00c200dd0015
:102c1000004d2100008040001000be00409588005b
:102c200051958800c9d2bf00caf2b700c972ec0042
:102c3000e5ff3900cb32a90000000600c1f2ef0029
:102c400000000600c552e20001003a004101070001
:102c5000c5f2ef0000000600c7f2ef00c8f2ef0077
:102c600000000600c6f2ef0000000600c3d2bf005d
:102c700080407800e1cf500005003a00c4d2bf0088
:102c80000080fb004300dd00e0948800eb0037008b
:102c9000c3d2bf0080407800e7cf50000a003a005e
:102ca000c4d2bf000080fb0000938800c4d2bf00e4
:102cb0000080fb0050938800c4d2bf000080fb005e
:102cc000a0938800dd003700c3d2bf0080407800a9
:102cd000efcf500011003a00c472ec000200200057
:102ce00003382400c4d2bf0048f707008bf6070062
:102cf00060958800719588006095800080958800b7
:102d0000709580009095880060958000a09588005f
:102d100070958000b0958800c8003700c3d2bf000e
:102d200080407800f1cf500007003a00c4d2bf00c5
:102d30005bf2b700d092800020938800d092800090
:102d400070938800bd003700c3d2bf008040780078
:102d5000f2cf500007003a00c4d2bf005ff2b700c4
:102d6000f092800040938800f09280009093880059
:102d7000b2003700c3d2bf0080407800f3cf5000cc
:102d800007003a00c452d40063f2b70010938000e9
:102d90006093880010938000b0938800a7003700ec
:102da000c3d2bf0080407800f5cf500054003a00f5
:102db00091928000c4d2bf000080fb00810f5000c0
:102dc0004e003200c452e20002003a002301070024
:102dd00047003700c4d2bf0080407800eccf5000dd
:102de00002003a008f01070041003700c4d2bf0043
:102df00080407800edcf500002003a00fa01070051
:102e00003b003700c4d2bf0080407800eecf5000b6
:102e100002003a006502070035003700c4d2bf0047
:102e200080407800efcf500002003a00d002070047
:102e30002f003700c4d2bf0080407800f0cf500090
:102e400002003a003b03070029003700c4d2bf004c
:102e500080407800f1cf500002003a00a60307003e
:102e600023003700c4d2bf0080407800f2cf50006a
:102e700002003a00110407001d003700c4d2bf0051
:102e800080407800f3cf500002003a007c04070035
:102e900017003700c4d2bf0080407800f4cf500044
:102ea00002003a00e704070011003700c4d2bf0057
:102eb00080407800f5cf500002003a00520507002c
:102ec0000b003700c4d2bf0080407800f6cf50001e
:102ed00002003a00bd05070005003700c4d2bf005c
:102ee00080407800f7cf500001003a002806070024
:102ef000c4d2bf000080fb00909288004f003700d2
:102f000020c4b300c352e30009003a00c452e200f7
:102f100004003a006900070010cea90014cea900f1
:102f20000200370010cea90014cea80043003700dd
:102f3000e0c4b300c352e30012003a0002002000d4
:102f400003302400c4d2bf00b0f60700f3f5070039
:102f50000200200003f0230091f50700209588006f
:102f60003195880022958000339580008092800002
:102f7000a7f607002cf6070060f6070050928800bd
:102f80002e003700f0c4b300c352e30012003a0031
:102f90000200200003302400c4d2bf009bf60700cb
:102fa000def507000200200003f023007cf5070097
:102fb0002095880031958800229580003395800007
:102fc0008092800092f6070017f607004bf6070084
:102fd000609288001900370000c5b300c352e300b7
:102fe00012003a000200200003302400c4d2bf00c7
:102ff00086f60700c9f507000200200003f0230051
:1030000067f507002095880031958800229580009b
:1030100033958000809280007df6070002f607005d
:1030200036f607007092880004003700b0c7b3007e
:10303000c352e30001003a0002000700c3f2ef00b0
:1030400000000600262cef00462cef00662cef0057
:103050002068a9002368a9002388a90015eea9000b
:1030600015aea900156ea900cc72ef00cd72ef006d
:10307000ce72ef00cb32a800c972ef0020c0b300bf
:10308000c952e3000a003e00c9d2bf000080fb0025
:10309000c200dd00004d210000814000f0ff2f0044
:1030a000f1ff2f000089be00c972ec00f3ff390068
:1030b00010aea90014aea90000000600cb32a80093
:1030c000c972ef0020c0b300c952e3000a003e00fd
:1030d000c9d2bf000080fb00c200dd00004d21000e
:1030e00000814000f0ff2f00f1ff2f000089be009b
:1030f000c972ec00f3ff3900262cef00462cef00dc
:10310000662cef002068a9002368a9002388a90085
:1031100011eea90015eea90011aea90015aea90087
:10312000116ea900156ea900cc72ef00cd72ef00f0
:10313000ce72ef00070007004a32ef004c32ef007a
:103140004e32ef004500070010aea90014aea900f2
:1031500000000600a0c0b3005bf2b70040c1b3009e
:103160005ff2b7006007200000938800a0c0b300a2
:1031700063f2b7004a32ef0060ec230070958800dc
:10318000ac32ef0000042000e0948800d092800070
:1031900020938800f0928000409388000093800084
:1031a0005093880010938000609388004c32ef00a9
:1031b00060958000809588007095800090958800cb
:1031c000d092800070938800f092800090938800e5
:1031d00000938000a093880010938000b093880033
:1031e0004e32ef0060958000a095880070958000b9
:1031f000b09588000000060010c0b300c9f2b70007
:10320000f0c7b300c952e30010003e00c9d2bf00ae
:10321000fef50700aaf407000001be0020852b0080
:103220005123240080f50700d9f50700912c2100d7
:10323000914078008180fb0081804000022d2100b8
:1032400080307900c972ec00edff390000202000c9
:10325000709e8800d032ef000000060080fa2d003a
:1032600000a3880060312d0010a3880080732c001b
:1032700020a3880060c02b0030a3880040172b00db
:1032800040a38800a0772a0050a38800f0e029001e
:1032900060a38800c052290070a3880080cc280059
:1032a00080a38800d04d280090a3880030d6270046
:1032b000a0a3880050652700b0a3880080fa2d00e5
:1032c000c0a3880060312d00d0a3880080732c003b
:1032d000e0a3880060c02b00f0a3880040172b00fb
:1032e00000a48800a0772a0010a48800f0e029003c
:1032f00020a48800c052290030a4880080cc280077
:1033000040a48800d04d280050a4880030d6270063
:1033100060a488005065270070a48800d0fa2600b9
:1033200080a488004096260090a48800503726008c
:10333000a0a48800c0dd2500b0a488003089250045
:10334000c0a4880060392500d0a4880000ee2400c5
:10335000e0a48800f0a62400f0a48800d063240034
:1033600000a588007024240010a58800b0e8230080
:1033700020a5880040b0230030a58800f07a230003
:1033800040a58800b048230050a5880030192300cc
:1033900060a5880070ec220070a5880020c2220081
:1033a00080a58800409a220090a588009074220091
:1033b000a0a5880000512200b0a58800702f22002f
:1033c000c0a58800d00f2200d0a58800e0f1210020
:1033d000e0a58800b0d52100f0a5880010bb210031
:1033e00000a68800e0a1210010a68800308a2100f4
:1033f00020a68800c073210030a68800a05e2100ae
:1034000040a68800b04a210050a68800d03721008d
:1034100060a688001026210070a68800d0b3ef00b7
:103420000000060080fa2d0000a38800801a2d00fd
:1034300010a38800506c2c0020a3880040a52b000e
:1034400030a38800d02d2b0040a38800a07a2a004a
:1034500050a3880050ef290060a388000050290085
:1034600070a38800b0ba280080a3880020612800db
:1034700090a38800e0c12700a0a388004072270025
:10348000b0a3880080fa2d00c0a38800801a2d0008
:10349000d0a38800506c2c00e0a3880040a52b002e
:1034a000f0a38800d02d2b0000a48800a07a2a0069
:1034b00010a4880050ef290020a4880000502900a3
:1034c00030a48800b0ba280040a4880020612800f9
:1034d00050a48800e0c1270060a488004072270043
:1034e00070a48800d0fa260080a48800d08a260024
:1034f00090a48800b0332600a0a4880030d0250016
:10350000b0a4880070942500c0a48800e03a25008b
:10351000d0a4880030f52400e0a4880090a5240001
:10352000f0a48800f05a240000a58800202e240072
:1035300010a5880080de230020a58800b0b62300f7
:1035400030a58800f07a230040a58800f0422300cf
:1035500050a588007017230060a58800a0e5220010
:1035600070a58800d0c7220080a58800009b22009b
:1035700090a5880020782200a0a588005050220045
:10358000b0a58800002b2200c0a58800a01422004e
:10359000d0a58800d0ec2100e0a58800e0d821006b
:1035a000f0a5880010bb210000a68800109f210014
:1035b00010a688004089210020a6880060702100a4
:1035c00030a688007061210040a68800104b2100c1
:1035d00050a68800a039210060a68800c0252100df
:1035e00070a6880000000600d0122e0000a38800fc
:1035f00060312d0010a38800f05d2c0020a388000e
:1036000090b92b0030a38800a0fd2a0040a38800b9
:10361000f08c2a0050a38800d0e3290060a3880022
:103620004060290070a38800f0c9280080a38800aa
:10363000003d280090a3880070e82700a0a3880020
:1036400020522700b0a38800d0122e00c0a388000b
:1036500060312d00d0a38800f05d2c00e0a388002d
:1036600090b92b00f0a38800a0fd2a0000a48800d8
:10367000f08c2a0010a48800d0e3290020a4880040
:103680004060290030a48800f0c9280040a48800c8
:10369000003d280050a4880070e8270060a488003e
:1036a0002052270070a488000007270080a488000b
:1036b0004096260090a48800902c2600a0a48800a4
:1036c00050da2500b0a48800607c2500c0a48800e2
:1036d00000442500d0a4880070ef2400e0a48800f6
:1036e000b0ad2400f0a488008062240000a588000a
:1036f000101c240010a58800d0f1230020a588000c
:10370000a0a6230030a588001081230040a58800d2
:10371000b048230050a58800d013230060a588007e
:10372000c0ea220070a58800c0bb220080a58800e6
:10373000909f220090a5880050752200a0a58800c7
:1037400060542200b0a58800d02e2200c0a58800b9
:10375000900b2200d0a5880070f62100e0a588001b
:10376000e0d02100f0a5880010be210000a688004e
:10377000e0a1210010a688008087210020a68800f3
:10378000f072210030a68800705b210040a68800fe
:10379000504d210050a688003038210060a68800d6
:1037a000c027210070a688000000060090022e00ad
:1037b00000a3880060482d0010a3880080732c00af
:1037c00020a3880000ac2b0030a38800d0102b0071
:1037d00040a38800705f2a0050a3880010f52900dc
:1037e00060a388007055290070a3880040d9280084
:1037f00080a38800604b280090a3880060c6270043
:10380000a0a3880090762700b0a3880090022e0025
:10381000c0a3880060482d00d0a3880080732c00ce
:10382000e0a3880000ac2b00f0a38800d0102b0090
:1038300000a48800705f2a0010a4880010f52900f9
:1038400020a488007055290030a4880040d92800a1
:1038500040a48800604b280050a4880060c6270060
:1038600060a488009076270070a48800b0e8260045
:1038700080a48800c0a1260090a4880050372600ac
:10388000a0a4880090d32500b0a48800f08525006e
:10389000c0a48800502d2500d0a4880010f8240072
:1038a000e0a4880040a82400f0a48800306a240026
:1038b00000a588004023240010a58800c0e0230054
:1038c00020a58800d0b8230030a58800e07123002f
:1038d00040a58800704e230050a5880030192300b1
:1038e00060a5880050e7220070a5880090c02200e3
:1038f00080a588003094220090a58800a07922003d
:10390000a0a58800b0512200b0a58800a0322200f6
:10391000c0a58800300f2200d0a58800f0ed21005e
:10392000e0a5880000da2100f0a5880080b621001b
:1039300000a68800c0a4210010a68800308a2100bb
:1039400020a688004071210030a68800d05d2100ab
:1039500040a68800a047210050a68800603a2100b8
:1039600060a688006026210070a68800000006007e
:10397000001b2e0000a3880000392d0010a3880032
:1039800040892c0020a3880060c02b0030a3880051
:1039900000042b0040a3880090712a0050a38800e7
:1039a00020ca290060a38800b065290070a38800a0
:1039b00010cf280080a38800e059280090a3880039
:1039c000f0d32700a0a3880060562700b0a388008a
:1039d000001b2e00c0a3880000392d00d0a3880052
:1039e00040892c00e0a3880060c02b00f0a3880071
:1039f00000042b0000a4880090712a0010a4880005
:103a000020ca290020a48800b065290030a48800bd
:103a100010cf280040a48800e059280050a4880056
:103a2000f0d3270060a488006056270070a48800a7
:103a3000100b270080a488002085260090a4880011
:103a400030422600a0a48800c0dd2500b0a4880074
:103a5000907f2500c0a4880050362500d0a488009f
:103a6000a0e22400e0a4880070b02400f0a4880044
:103a70001065240000a58800802a240010a5880075
:103a800080e7230020a58800c0a8230030a5880077
:103a90001083230040a588002040230050a5880003
:103aa000a01e230060a5880070ec220070a588008d
:103ab00050bd220080a58800c098220090a58800f3
:103ac000e06e2200a0a58800c0552200b0a58800a5
:103ad00020302200c0a58800d0122200d0a5880086
:103ae00050f12100e0a58800f0d12100f0a5880068
:103af00020bf210000a68800a09d210010a68800fc
:103b0000e08c210020a68800c073210030a6880028
:103b1000405c210040a68800f049210050a68800a2
:103b20000035210060a688007028210070a688005a
:103b30000000060040de2d0000a3880010502d007c
:103b400010a38800c07a2c0020a38800d0d42b00ba
:103b500030a3880040172b0040a3880080652a000e
:103b600050a3880030db290060a38800303d290085
:103b700070a3880070de280080a3880030502800e1
:103b800090a38800a0e12700a0a38800306327004d
:103b9000b0a3880040de2d00c0a3880010502d0087
:103ba000d0a38800c07a2c00e0a38800d0d42b00da
:103bb000f0a3880040172b0000a4880080652a002d
:103bc00010a4880030db290020a48800303d2900a3
:103bd00030a4880070de280040a4880030502800ff
:103be00050a48800a0e1270060a48800306327006b
:103bf00070a48800b0ec260080a4880090a5260060
:103c000090a4880030272600a0a4880000e82500a2
:103c1000b0a4880030892500c0a488005030250059
:103c2000d0a4880030eb2400e0a48800309c24005d
:103c3000f0a48800c06c240000a58800b0252400f2
:103c400010a5880060ee230020a5880020af230087
:103c500030a58800e073230040a588006050230051
:103c600050a588002011230060a5880090f1220053
:103c700070a5880020c2220080a58800b09522008f
:103c800090a5880020732200a0a58800a04b2200e8
:103c9000b0a58800f0332200c0a588006010220083
:103ca000d0a58800c0f42100e0a5880020d521001f
:103cb000f0a5880080b7210000a68800c0a52100db
:103cc00010a688002086210020a6880050762100ba
:103cd00030a68800a05e210040a688007048210020
:103ce00050a688002037210060a6880060232100ac
:103cf00070a688000000060070f62d0000a3880062
:103d0000c0162d0010a3880080902c0020a38800ee
:103d100030c72b0030a38800902a2b0040a38800d6
:103d2000a0772a0050a38800d0cf290060a3880084
:103d3000504d290070a3880030b8280080a3880067
:103d4000b05e280090a3880080d82700a0a3880038
:103d500010702700b0a3880070f62d00c0a3880063
:103d6000c0162d00d0a3880080902c00e0a388000e
:103d700030c72b00f0a38800902a2b0000a48800f5
:103d8000a0772a0010a48800d0cf290020a48800a2
:103d9000504d290030a4880030b8280040a4880085
:103da000b05e280050a4880080d8270060a4880056
:103db0001070270070a48800c0f8260080a4880036
:103dc000f088260090a48800d0452600a0a4880092
:103dd00080ce2500b0a48800d0922500c0a4880021
:103de00060392500d0a4880070e52400e0a4880094
:103df00040a42400f0a48800a059240000a5880055
:103e0000f02c240010a58800d0e9230020a588000c
:103e1000a0b5230030a58800f079230040a58800d4
:103e20000042230050a588007020230060a5880070
:103e3000d0e4220070a5880000c7220080a5880079
:103e4000409a220090a5880050702200a0a588000a
:103e5000b04f2200b0a58800602a2200c0a58800cb
:103e600000142200d0a5880070f22100e0a588008f
:103e700060d82100f0a5880080ba210000a6880043
:103e8000909e210010a68800d08d210020a68800d9
:103e9000f06f210030a688001061210040a6880044
:103ea000b04a210050a68800b035210060a68800e5
:103eb0006025210070a688000000060050e62d0055
:103ec00000a38800902d2d0010a38800605a2c00bc
:103ed00020a38800b0db2b0030a38800b01d2b008e
:103ee00040a38800e0892a0050a38800f0e0290060
:103ef00060a388009042290070a3880060c7280052
:103f000080a38800a03a280090a3880030e627000c
:103f1000a0a3880080672700b0a3880050e62d008a
:103f2000c0a38800902d2d00d0a38800605a2c00db
:103f3000e0a38800b0db2b00f0a38800b01d2b00ad
:103f400000a48800e0892a0010a48800f0e029007d
:103f500020a488009042290030a4880060c728006f
:103f600040a48800a03a280050a4880030e627002a
:103f700060a488008067270070a48800f0042700f0
:103f800080a488005094260090a48800c02a2600af
:103f9000a0a4880060eb2500b0a48800d07a25009a
:103fa000c0a4880080422500d0a4880000ee240030
:103fb000e0a48800d09e2400f0a488004061240082
:103fc00000a58800e01a240010a58800a0f02300b6
:103fd00020a5880050b1230030a588000080230070
:103fe00040a58800c047230050a58800f012230098
:103ff00060a5880040f3220070a58800f0ba220076
:1040000080a58800d09e220090a588009074220090
:10401000a0a58800004d2200b0a58800302e220007
:10402000c0a58800000b2200d0a58800e0f5210083
:10403000e0a5880030d62100f0a5880090bd2100c1
:1040400000a6880070a1210010a68800008721002a
:1040500020a688003077210030a68800105b210060
:1040600040a68800f04c210050a68800d0372100df
:1040700060a688001024210070a6880000000600b9
:1040800080fe2d0000a38800501e2d0010a3880084
:10409000f06f2c0020a38800a0a82b0030a388007c
:1040a00010312b0040a38800b07d2a0050a3880067
:1040b00030f2290060a38800c052290070a3880054
:1040c00040bd280080a388000049280090a38800f4
:1040d00020c42700a0a3880060742700b0a3880034
:1040e00080fe2d00c0a38800501e2d00d0a38800a4
:1040f000f06f2c00e0a38800a0a82b00f0a388009c
:1041000010312b0000a48800b07d2a0010a4880084
:1041100030f2290020a48800c052290030a4880071
:1041200040bd280040a488000049280050a4880011
:1041300020c4270060a488006074270070a4880051
:10414000d0fc260080a48800d09f260090a4880080
:1041500080352600a0a48800e0d12500b0a4880006
:1041600010962500c0a48800d02b2500d0a488007c
:10417000a0f62400e0a48800f0a62400f0a48800a3
:10418000305c240000a588001022240010a58800bf
:10419000a0df230020a58800c0b7230030a5880039
:1041a000f07b230040a58800704d230050a58800b7
:1041b0005018230060a5880080e6220070a58800c2
:1041c000a0c8220080a588007093220090a58800d6
:1041d000e0782200a0a5880000512200b0a5880048
:1041e000a02b2200c0a58800900e2200d0a5880038
:1041f00060ed2100e0a5880070d92100f0a58800bd
:1042000090bb210000a6880050a4210010a68800c1
:10421000b089210020a68800d070210030a6880037
:10422000e061210040a688004047210050a6880098
:10423000003a210060a688001026210070a68800a0
:1042400000000600f0162e0000a3880030352d0077
:1042500010a3880090612c0020a38800f0bc2b00e4
:1042600030a38800d0002b0040a38800f08f2a00e4
:1042700050a38800b0e6290060a3880000632900ed
:1042800070a3880080cc280080a38800603f2800ad
:1042900090a38800b0d12700a0a388004054270035
:1042a000b0a38800f0162e00c0a3880030352d0082
:1042b000d0a3880090612c00e0a38800f0bc2b0004
:1042c000f0a38800d0002b0000a48800f08f2a0003
:1042d00010a48800b0e6290020a48800006329000b
:1042e00030a4880080cc280040a48800603f2800cb
:1042f00050a48800b0d1270060a488004054270053
:1043000070a488000009270080a488002098260057
:1043100090a4880060402600a0a4880000dc25004e
:10432000b0a48800007e2500c0a488009045250028
:10433000d0a4880030e12400e0a4880010af24005d
:10434000f0a48800d063240000a58800401d24004c
:1043500010a5880060e6230020a58800b0a72300f0
:1043600030a588001082230040a58800a0492300c2
:1043700050a58800c01d230060a5880090eb220096
:1043800070a5880090bc220080a5880050a0220063
:1043900090a58800306e2200a0a58800105522004c
:1043a000b0a58800702f2200c0a58800300c220024
:1043b000d0a58800c0f02100e0a5880060d12100d0
:1043c000f0a5880090be210000a6880060a2210010
:1043d00010a68800708c210020a688005073210050
:1043e00030a68800d05b210040a68800b04d210097
:1043f00050a68800a034210060a688002028210053
:1044000070a688000000060040da2d0000a3880096
:10441000304c2d0010a3880020772c0020a38800aa
:1044200060af2b0030a3880000142b0040a388004d
:1044300070622a0050a38800f0f7290060a388006a
:104440002058290070a38800d0db280080a38800b2
:10445000d04d280090a38800a0c82700a0a3880002
:1044600010612700b0a3880040da2d00c0a38800a7
:10447000304c2d00d0a3880020772c00e0a38800ca
:1044800060af2b00f0a3880000142b0000a488006c
:1044900070622a0010a48800f0f7290020a4880088
:1044a0002058290030a48800d0db280040a48800d0
:1044b000d04d280050a48800a0c8270060a4880020
:1044c0001061270070a48800b0ea260080a488004c
:1044d000b0a3260090a4880020392600a0a488005c
:1044e00040e62500b0a4880090872500c0a488007d
:1044f000d02e2500d0a4880080f92400e0a48800f4
:10450000d09a2400f0a48800806b240000a58800c5
:104510007024240010a58800e0e1230020a5880075
:1045200010ae230030a58800e072230040a588006b
:10453000604f230050a58800201a230060a5880042
:10454000b0f0220070a5880050c1220080a588002c
:10455000f094220090a58800507a2200a0a588003f
:10456000f04a2200b0a5880050332200c0a5880080
:10457000d00f2200d0a5880080ee2100e0a58800a1
:10458000a0d42100f0a5880000b7210000a6880073
:1045900040a5210010a68800a08a210020a688003e
:1045a000e075210030a68800405e210040a688000a
:1045b0000048210050a68800b03a210060a688007b
:1045c0001023210070a6880000000600101f2e0096
:1045d00000a38800f0122d0010a38800e08c2c00ae
:1045e00020a38800c0c32b0030a3880030072b0015
:1045f00040a3880090742a0050a3880000cd2900b1
:1046000060a388007068290070a38800a0d12800ea
:1046100080a38800405c280090a3880030d6270043
:10462000a0a3880080582700b0a38800101f2e0088
:10463000c0a38800f0122d00d0a38800e08c2c00cd
:10464000e0a38800c0c32b00f0a3880030072b0034
:1046500000a4880090742a0010a4880000cd2900ce
:1046600020a488007068290030a48800a0d1280008
:1046700040a48800405c280050a4880030d6270061
:1046800060a488008058270070a48800c0f6260027
:1046900080a488000087260090a48800004426009b
:1046a000a0a4880070df2500b0a4880040912500f8
:1046b000c0a48800d0372500d0a4880010e42400ce
:1046c000e0a48800c0b12400f0a488006058240051
:1046d00000a58800b02b240010a58800b0e82300b6
:1046e00020a58800d0a9230030a58800f0782300f9
:1046f00040a588001041230050a58800901f23008a
:1047000060a5880040ed220070a5880030c6220018
:1047100080a588008099220090a58800906f2200d3
:10472000a0a5880070562200b0a58800c0292200ec
:10473000c0a5880060132200d0a58800e0f1210008
:10474000e0a5880070d22100f0a5880000ba210001
:1047500000a68800109e210010a68800508d210020
:1047600020a688003074210030a68800a0602100b7
:1047700040a68800504a210050a6880060352100dc
:1047800060a68800c028210070a6880000000600ee
:1047900040e22d0000a38800f0532d0010a38800f4
:1047a000d0562c0020a3880040d82b0030a38800ce
:1047b000701a2b0040a3880080682a0050a388004c
:1047c00010de290060a38800e03f290070a3880064
:1047d00000e1280080a38800a052280090a3880050
:1047e000e0e32700a0a3880050652700b0a388005d
:1047f00040e22d00c0a38800f0532d00d0a3880014
:10480000d0562c00e0a3880040d82b00f0a38800ed
:10481000701a2b0000a4880080682a0010a4880069
:1048200010de290020a48800e03f290030a4880081
:1048300000e1280040a48800a052280050a488006d
:10484000e0e3270060a488005065270070a488007a
:10485000b0ee260080a488007092260090a4880004
:10486000f0282600a0a48800b0e92500b0a48800a4
:10487000c08a2500c0a48800f0402500d0a488008c
:1048800090ec2400e0a48800809d2400f0a488001f
:10489000106e240000a58800b019240010a588001f
:1048a00080ef230020a5880040b0230030a58800b9
:1048b000e074230040a58800c046230050a588006e
:1048c0001012230060a5880060f2220070a5880005
:1048d000f0c2220080a58800109e220090a58800ca
:1048e000e0732200a0a58800504c2200b0a58800eb
:1048f00090342200c0a58800600a2200d0a588005c
:1049000050f52100e0a58800b0d52100f0a5880071
:1049100000b8210000a68800f0a0210010a68800a1
:104920009086210020a68800c076210030a688004d
:10493000005f210040a68800904c210050a688000e
:104940008037210060a68800b023210070a688006f
:0849500000000600ffff370024
:020000040000fa
:104958001a12000014000000800000002e1200004f
:104968007200000080000000a01200001800000083
:1049780080000000b812000018000000800000004d
:10498800d01200000002000080000000d0140000d7
:104998000c00000080000000dc1400000001000092
:0849a800800000000000000087
:00000001FF
